:020000000F28C7
:080008000B110900F6000030A5
:100010008A000F30760703188A0A76088207203094
:1000200083120313BB000430BC000230BD00D701B3
:1000300083120313D8010930D9000230DA000130ED
:10004000DB000230DC000830DD000330DE0004306D
:100050008600F03083168500F23086004030810043
:100060008B01F3260730831203139F001930831688
:100070009900243098009030831298008C01B701C9
:100080000130B600B901B8013030CA006927B701A4
:100090000230B600B901B8014030CA006927FA3011
:1000A000B400A627FA30B400A627FA30B400A62779
:1000B000302783120313B7010230B600B901B8012B
:1000C000CA016927FC24FC24831203130608F000EC
:1000D000F00CF00CF00C700C0F39F0007008063CBE
:1000E000031D7C2883120313A001A101A201A30117
:1000F0008F30A400E124F6297008073C031DDF2897
:100100000130831203135B02031DB6280530580229
:10011000013003180301F1005808073C01300318AF
:1001200003017104003C0319AF285808093C013051
:1001300003190301F10058080B3C013003190301B6
:100140007105003C0319AF285808A000A101A201C5
:10015000A3010730A400E12483120313CC00D80AC2
:100160000D305802031DF629D801F62902308312FA
:1001700003135B02031DC52806305E02031DC3285E
:100180000130DE00DE28DE0ADE280330831203138E
:100190005B02031DDE28A001A101A201A3015D08ED
:1001A000A400E12483120313CC0008305D02031D78
:1001B000DC288830DD00DE280830DD00F6297008F4
:1001C0000B3C031D64290130831203135B02031DE2
:1001D000422901305002031D0929F1015508103E42
:1001E0000318F10AD500F100F10CF10CF10C710CBF
:1001F0000F390E3C031D24295508F100710EF0390A
:10020000F039F100F10CF10CF10C710C0F39D50043
:100210002429F101831203135508013E0318F10A42
:10022000D500F100710EF039F039E03C031D2429AE
:100230005508F100F10CF10CF10C710C0F39F100C3
:10024000710EF039F039D500CB01C4275930831233
:100250000313CB00C427831203135508CB00C42714
:10026000831203135608CB00C427BC308312031338
:10027000CB00C427D32783120313CC000A30B40069
:10028000A627F62902305B02031D4B29C2015E0836
:10029000C3003C2563290330831203135B02031D53
:1002A0006329A001A101A201A3015C08A400E1242B
:1002B00083120313CC00CC08031D61298230DC00BB
:1002C00063290230DC00F62970080D3C031DB129BA
:1002D0000130831203135B02031D7929A001A101E0
:1002E000A201A3018130A400E12483120313CC00F6
:1002F000F62902305B02031D83290130C2005E082B
:10030000C3003C25B0290330831203135B02031D95
:10031000B02954080C3C0130031D0301F1005408BE
:10032000C03C0130031D03017104003C0319B029D6
:100330005908A000A101A201A3010930A400E124F1
:1003400083120313CC0089305902031DAA290930F6
:10035000D900B029F1015908403E0318F10AD9002B
:10036000F62970080E3C031DF6290430831203138E
:100370005A02031DBD290130DA003230B400A6272D
:100380005A08F1007108013C031DD229831203139E
:10039000B7010230B600B901B801CA0169270130BE
:1003A000DB00F4297108023C031DE32983120313C7
:1003B000B7010230B600B901B8011030CA00692790
:1003C0000230DB00F4297108033C031DF429831279
:1003D0000313B7010230B600B901B8012030CA00DA
:1003E00069270330DB00F429DA0AF629FC24CB0163
:1003F000C427593083120313CB00C427831203137D
:10040000CB01C42783120313CB01C427BB30831253
:100410000313CB00C427D32783120313D500D3279C
:1004200083120313D600CB01C42755308312031364
:10043000CB00C42783120313CB01C42783120313F9
:10044000CB01C427BB3083120313CB00C427D327AF
:10045000FE00D327FF007E088039003C03196C2A78
:100460007E08F0007008813C031D3D2A4230831253
:100470000313D3000130D000772A7008803C031D9D
:10048000472A413083120313D300D001772A700822
:10049000903C031D4C2A502A7008913C031D532A9E
:1004A0004830D300772A7008843C031D582A5C2A00
:1004B0007008853C031D5F2A5130D300772A7008ED
:1004C000863C031D642A682A7008873C031D6B2A3A
:1004D0007430D300772A772A4D3083120313D30068
:1004E0007E082039003C0319772A5430D3000130AC
:1004F000BF00C0015308C1002E25F0013030F100CB
:10050000831203132508F200F20CF20CF20C720CA9
:100510000F3971070318F00AAA00303C031D922A14
:100520002030AA00F0013030F1002508F200720EF0
:10053000F039F039F200F20CF20CF20C720C0F39B7
:1005400071070318F00AAB002A08203C0130031D94
:100550000301F0002B08303C0130031D030170053E
:10056000003C0319B52A2030AB00F0013030F10017
:100570002608F200F20CF20CF20C720C0F39710723
:100580000318F00AAC002E30AD00F0013030F1005D
:100590002608F200720EF039F039F200F20CF20C7B
:1005A000F20C720C0F3971070318F00AAE00F0015B
:1005B0003030F1002708F200F20CF20CF20C720C51
:1005C0000F3971070318F00AAF00F0013030F10065
:1005D0002708F200720EF039F039F200F20CF20C3A
:1005E000F20C720C0F3971070318F00AB0002E30AC
:1005F000B100F0013030F1002808F200F20CF20CEA
:10060000F20C720C0F3971070318F00AB200F001F6
:100610003030F1002808F200720EF039F039F200A3
:10062000F20CF20CF20C720C0F3971070318F00A7D
:10063000B3005708093C031C322B0130BF00F00106
:10064000023057070318F00AC00057082A3E8400FA
:100650008313000883120313C1002E258312031392
:10066000D70A192BD7015708023C031C5B2B01301A
:10067000BF00F0010D3057070318F00AC000290829
:10068000F7000330F800EF27F0007808583EF1003B
:100690000318F00A7108831203135707F1000318B7
:1006A000F00A7108BE0026258312C1002E25831290
:1006B0000313D70A332BD70101305002031D6D2BD2
:1006C0000330D1003C30D2005508F000F00CF00CA3
:1006D000F00C700C0F39D400772B0130D100B630FC
:1006E000D2005508F000700EF039F039D4005408EB
:1006F0000C3C0130031D0301F0005408C03C0130E4
:10070000031D03017004003C0319B42B5108CB00F6
:10071000C427831203135208CB00C4278312031388
:10072000CB01C42783120313CB01C427BB30831230
:100730000313CB00C427D327FE00D327FF007E0876
:10074000643C031DA82B2D3083120313D300B82B58
:100750007E08A43C031DB12B2B3083120313D3005E
:10076000B32B2030D300B82B203083120313D300D7
:100770000130BF000C30C0005308C1002E25831289
:100780000313CB01C427793083120313CB00C42792
:1007900083120313CB01C42783120313CB01C42795
:1007A000BB3083120313CB00C427D327FE00D3270B
:1007B000FF007E08F000700EF039F039F00070088C
:1007C000003C031DE42BE82B7008403C031DED2B7F
:1007D000343083120313D300132C7008103C031D14
:1007E000F22BF62B7008503C031DFB2B3330831289
:1007F0000313D300132C7008203C031D002C042C81
:100800007008603C031D072C3230D300132C700895
:10081000303C031D0C2C102C7008703C031D132C55
:100820003130D300132C0230BF000530C000530814
:10083000C1002E257F088039003C03192D2C033080
:10084000831203135B02031D362C0230BF000C30F1
:10085000C0002A30C1002E25362C0230831203132B
:10086000BF000C30C0002030C1002E2583120313BE
:10087000A001A101A201A301F730A400E124831289
:100880000313CC008039031D612C0230BF00C0016E
:100890005030C1002E25831203134C1F572C0230F9
:1008A000BF000330C0004830C1002E25832C023029
:1008B00083120313BF000330C0004C30C1002E254B
:1008C000832C83160313051602308312BF00C00168
:1008D0007330C1002E2583120313A001A101A201D0
:1008E000A301E730A400E12483120313CC00803974
:1008F000031D832C8316051202308312BF00C00132
:100900005330C1002E25831203134C08F000700EE3
:10091000F039F039F000F00CF00CF00C700C0F39DD
:10092000CD0001304D02031CB22C01304D020130CC
:10093000031C0301F0004D08093C0130031C0301B6
:100940007005003C0319AD2CF00130304D07031841
:10095000F00ACE002030CF00B72C3930CE002B303B
:10096000CF00B72C203083120313CE00CF0002300B
:10097000BF000130C0004E08C1002E250230831296
:100980000313BF00C0004F08C1002E2502308312A0
:1009900003135B02031DD72C0230BF000F30C000D1
:1009A000F00130305E070318F00AC1002E25023036
:1009B00083120313BF000630C0007C30C1002E2517
:1009C0006428831203132008CB00C4278312031367
:1009D0002108CB00C427831203132208CB00C427AD
:1009E000831203132308CB00C427831203132408A4
:1009F000CB00C427D327080083120313CB01C427DD
:100A000083120313CB01C42783120313CB01C42722
:100A100083120313CB01C427033083120313CB00CB
:100A2000C427D32783120313A500D32783120313EC
:100A3000A600D32783120313A700D327831203131F
:100A4000A800D32783120313A900080083120313FD
:100A50003E0883169B001C141A0808008312031317
:100A60003F08C8004008C9003C278312031306143E
:100A70004108C70019270800303083120313E10032
:100A80003930E2004208003C03194B2D6208DF00B8
:100A90006108E0004F2D6108DF006208E0004308B4
:100AA000063C031C832E33085F020130031D030143
:100AB000F100023043020130031C0301F20043083D
:100AC000063C0130031C030172057104003C03194C
:100AD000782E01304302031D6F2D6008B3003208E9
:100AE0005F020130031D0301F100033043020130B6
:100AF000031C0301F2004308063C0130031C030100
:100B000072057104003C03196D2E4308013C01304D
:100B1000031D0301F1004308023C0130031D0301E2
:100B20007104003C0319962D6008B20030085F0282
:100B30000130031D0301F100043043020130031CA6
:100B40000301F2004308063C0130031C0301720557
:100B50007104003C03195B2E013043020130031C79
:100B60000301F1004308033C0130031C030171053C
:100B7000003C0319BD2D6008B0002F085F02013052
:100B8000031D0301F100053043020130031C030182
:100B9000F2004308063C0130031C03017205710496
:100BA000003C0319502E013043020130031C0301A5
:100BB000F1004308043C0130031C03017105003CB3
:100BC0000319E42D6008AF002E085F020130031DF9
:100BD0000301F1004308063C0130031D03017104C9
:100BE000003C0319452E013043020130031C030170
:100BF000F1004308053C0130031C03017105003C72
:100C00000319042E6008AE002C085F02031D3A2E63
:100C1000013043020130031C0301F1004308063C8C
:100C20000130031C03017105003C0319192E6008F3
:100C3000AC002B085F02031D2F2E6008AB002A08B2
:100C40005F02031D262E6008AA00832E2A08C40016
:100C50004208C5000130C600E126AA00832E831297
:100C600003132B08C4004208C5000130C600E1266A
:100C7000AB00832E831203132C08C4004208C50066
:100C80000130C600E126AC00832E831203132E0828
:100C9000C4004208C5000130C600E126AE00832E24
:100CA000831203132F08C4004208C5000130C60098
:100CB000E126AF00832E831203133008C4004208DC
:100CC000C5000130C600E126B00003304302031D19
:100CD0006C2E3030B200B300832E8312031332081F
:100CE000C4004208C5000130C600E126B200832ED0
:100CF000831203133308C4004208C5000130C60044
:100D0000E126B300832EF101831203132A08F200B7
:100D1000720EF039F039F2002B08F300730EF0393F
:100D2000F039F300F30CF30CF30C730C0F3972076A
:100D30000318F10AA000F1012C08F200720EF0393C
:100D4000F039F2002E08F300730EF039F039F30099
:100D5000F30CF30CF30C730C0F3972070318F10A40
:100D6000A100F1012F08F200720EF039F039F20003
:100D70003008F300730EF039F039F300F30CF30C84
:100D8000F30C730C0F3972070318F10AA200F1017A
:100D90003208F200720EF039F039F2003308F30035
:100DA000730EF039F039F300F30CF30CF30C730C01
:100DB0000F3972070318F10AA3000130A400E124DF
:100DC0000800831203134508003C0319EE2EF101BD
:100DD000440846070318F10AC400F12E46084402ED
:100DE000C40044080800831203138611061005305E
:100DF000B400A627033085002B270530B400A627B2
:100E0000023085002B270530B400A6272830C70004
:100E10001927083083120313C70019270C308312D7
:100E20000313C7001927063083120313C7001927BD
:100E30000800831203134708F300F30CF30CF30CC0
:100E4000730C0F3985002B27470885002B27283086
:100E5000BA00B7270800831203138615861108000D
:100E60008312031306100130C700192702308312C2
:100E70000313B400A62708008312031306104808C2
:100E8000F2007208013C031D4F2FF30180308312E2
:100E9000031349070318F30AC7001927632F7208C1
:100EA000023C031D632FF3014030831203134907F3
:100EB0000318F30AF40073080038F300740880384C
:100EC000C7001927632F023083120313B400A6272B
:100ED000080083120313DF01E0016008003C0030CA
:100EE000031C7A2F0130031D7A2F5F080F3C01305D
:100EF000031C0301003C0319A52F3708F200360834
:100F0000C8003908F2006008F20738085F070318C4
:100F1000F20AC9003C278312031306140030F200C2
:100F20006008F2074A085F070318F20ABE00262588
:100F3000013CF2007209013E8312C7001927831297
:100F40000313DF0A0319E00A6D2F08008E308312A5
:100F50000313B500000000000000000000000000C6
:100F6000B50BAC2F0000B40BA62F000008008312B5
:100F70000313BA0CBA0C3F30BA050330BA020000B2
:100F8000BA0BBF2F00000800831203134B0899000F
:100F900083168312031301080319D12F831618082F
:100FA000C92F83120800831203130C083B05FF3975
:100FB000003C0319D32F18083C05FF39F10018082D
:100FC0003D05FF397104003C0319EB2F1812000096
:100FD00018161A08E3001A080800D32F0800093071
:100FE000F9007708F7010310F70CF80C0318F7075E
:080FF000F90BF42F770808004B
:02400E00503F21
:104200002100210021002100210021002100570070
:10421000670021004300650021004E006500210079
:104220002100210021002100210021002100560051
:104230007100210045007800210054007500210024
:104240002100210021002100210021002100530034
:10425000710021005400710021005100550021001F
:10426000470055002E00390032003800210053006D
:1042700066006E007000750066004E0062006F0000
:104280004A00580033004D004700450021007300EC
:1042900032002F003300210033003100310036009E
:1042A00020002000720031002E0032002E0032006B
:1042B0004C005300420055005300420020004300D0
:1042C0005700430057005200200041004D000000FD
:1042D00000000000570046004D00000000000000F4
:1042E000200046004D00000000000000440049008E
:1042F000470000000000000050004B005400000088
:00000001FF
